:10000000A729910192011130930010080E06940067
:100010008E1F14288E098D098D0A03198E0A9308E4
:10002000031D14280D080800901F1B2890098F0934
:100030008F0A0319900A2B28910D920D0F081102B7
:100040001008031C100F1202031827282B289200F7
:100050000F08910203148D0D8E0D93039308031D59
:100060001C28941F34280A280D0808009200120842
:100070009D00F93084000000840B3B289D0B39283B
:1000800008008F000F089D00193084000000840BC9
:1000900046289D0B442808000000000000000000D6
:1000A0000000000008005C20AC306C20083092207A
:1000B000961F5B2808005328831205120630412042
:1000C00005164C208312051E662862288312051A25
:1000D0006A286628063041288D0001309E009F0165
:1000E00008301F02031891280D081E05003A031D51
:1000F0008528831205124C204C204C204C204C208B
:100100004C204C204C204C208928831205120000E2
:100110000000831205160130412003109E0D9F0A36
:10012000702808008D0001309E008E019F0108306C
:100130001F020318B72883120512000000000516DD
:1001400000000000000000000000000000000000AF
:10015000051EAD281E088E04B1288312051AB12889
:10016000AD280130412003109E0D9F0A97280E08EC
:10017000960097010D08093A031DD3288312051232
:100180000000000005160000000000000000000054
:10019000000000000000051ECF28970AD328831214
:1001A000051AD328CF2806304128031010308D00BF
:1001B0009A019B019C01980D990D9C0D9B0D9A0D28
:1001C0008D0BE32808001C308400EE201B308400D7
:1001D000EE201A308400EE20DB28080003300007F0
:1001E0008E008E198000303000078E008E1B80003C
:1001F00008008D000D0E0F398E000A300E02031814
:10020000042930308E07062937308E070E08162154
:100210000F300D058E000A300E02031812293030FF
:100220008E07142937308E070E0816299000831286
:1002300006089500951215088600100E0F399100DA
:10024000F03095051108950495161508860095124D
:10025000150886000F3010059100F0309505110843
:10026000950495161508860095121508860001302C
:1002700036288E0015121508831286000D08013AE3
:1002800003194629033A03194A294E297F300E07DC
:100290008F004F29BF300E078F004F294F290F08BD
:1002A00016211516150883128600053036281512FA
:1002B00015088312860001301621151615088312C1
:1002C000860005303628151215088312860095120F
:1002D00015088600FF3036208D018D1B73290330F1
:1002E0000D0203188429F030950503309504150894
:1002F000831286009516150886009512150886004B
:10030000643036208D0A6D2902309500150883125D
:1003100086009516150886000530362028301621EF
:100320000530362014301621053036200C301621C9
:1003300005303620063016210530362002301621D1
:100340000530362015161508831286000800D630B1
:10035000831681000F3085004030860040308312C4
:1003600086001F308500632157215C200C306C20F3
:1003700041306C20FF303620D430A7003030A80048
:100380008430A900EA30AA005C20EE306C205320B3
:100390005C20AA306C20083092201608A0005C2057
:1003A000A0306C20093092201608A3001708A40082
:1003B0005C2041306C205C20A0306C200930922001
:1003C0001608A5001708A600A01FE829A003A00A88
:1003D0002008A100A201A11BA20321089600220867
:1003E00097008C0163300C020318FE291708A2073E
:1003F0001608A1070318A20A8C0AF229A61B2B2AA9
:100400002508260403192B2A24082602A400230801
:100410002502A300031CA4032308960024089700C8
:100420008C0163300C0203181D2A1708A407160854
:10043000A3070318A40A8C0A112A23088D00240894
:100440008E0025088F002608900001200D08A300CB
:100450000E08A4002E2A3230A300A4012408A2070B
:100460002308A1070318A20A3230A102031CA20329
:10047000210896002208970001308D0001303921B3
:1004800086222808220203194D2A2808220603186A
:10049000803A80390319512A552A27082102031866
:1004A000552A2108A7002208A80022082A020319B9
:1004B000612A2A0822060318803A80390319652A1E
:1004C000692A210829020318692A2108A90022089B
:1004D000AA0083128519712A270896002808970018
:1004E000752A290896002A08970002308D000130ED
:1004F0003921862283120519852AD430A70030308D
:10050000A8008430A900EA30AA00C429971F902AC5
:1005100097099609960A0319970A2D301621922AEF
:100520002B3016211708990016089800D520303076
:100530001A0716211B08F9202E3016211C08F92055
:04054000DF30162969
:02400E00F13F80
:00000001FF
